:1000000000308A00F12C0000FF00030E8301A100E4
:100010000A08A0008A010408A2007708A300780853
:10002000A4007908A5007A08A6007B08A70083131E
:1000300083120B1E1D288B183028220884002308E9
:10004000F7002408F8002508F9002608FA00270818
:10005000FB0020088A00210E8300FF0E7F0E09009E
:100060008A110A12302C0A108A100A1182074834A9
:1000700065346C346C346F34203457346F347234DC
:100080006C34643421340D340A3400340A108A107C
:100090000A1182071B345B3432344A3400340A10AC
:1000A0008A100A11820750347534743474346934F8
:1000B0006E3467342034703469346E3473342034D1
:1000C00069346E3474346F3420346B346E346F346E
:1000D00077346E342034733474346134743465345A
:1000E000203461346E3464342034723465347334B3
:1000F00065347434743469346E3467342034443471
:10010000313432340D340A3400340A108A100A11A2
:1001100082071B345B3431346D34523465346134BE
:10012000643479341B345B3430346D342E342034F1
:1001300050347234653473347334203461346E3423
:10014000793420346B3465347934203474346F342A
:100150002034703472346F346334653465346434FD
:100160002E340D340A3400340A108A100A11820722
:1001700043344D3444343A342034203453346534D9
:1001800074342034413464346434723465347334E8
:1001900073342F3445346E34613462346C346534D6
:1001A0000D340A3400340A108A100A118207093407
:1001B00044344134543441343A3420343034783483
:1001C000383430342034283445346E346134623469
:1001D0006C3465342C3420346E346F342034613404
:1001E00064346434723465347334733429340D34B4
:1001F0000A34003400000A148A100A11023E03185F
:100200008A0A820043344D3444343A342034203452
:10021000533465347434203465346E34643470344B
:100220006F3469346E347434203465346E34613420
:1002300062346C3465340D340A3400340A148A1084
:100240000A118207093444344134543441343A3475
:100250002034303478343034313420342834453448
:100260006E34613462346C346534643429340D3452
:100270000A3400340A148A100A11820743344D34B8
:1002800044343A34203420345334653474342034C4
:100290004D346F34643465340D340A3400340A1438
:1002A0008A100A11820709344434413454344134E9
:1002B0003A3420344E346F3420344C3461347A3440
:1002C0007934203443346C346F3463346B342C34DD
:1002D000203443346C346F3463346B342034523400
:1002E00075346E346E3469346E3467342C34203493
:1002F00000340A148A100A11820749346E347434A7
:1003000065347234723475347034743473343D34FB
:1003100031342C34203453346F34663474344334E1
:100320006F346E346E346534633474343D34313438
:100330000D340A3400340A148A100A118207093471
:1003400044344134543441343A34203453347434D2
:1003500061347234743420346F346634203446345B
:10036000723461346D346534203469346E347434DD
:1003700065347234723475347034743420346434B7
:1003800069347334613462346C34653464342C34CD
:10039000203400340A148A100A1182075334653459
:1003A00074342D3474346F342D346F346E346534BA
:1003B00020346E346F3474342034733465347434C0
:1003C0002C34203400340A148A100A11EA3E03182F
:1003D0008A0A82000D340A340934093443346C34F7
:1003E0006F3463346B342034443469347634693484
:1003F000733469346F346E3420344634613463347A
:1004000074346F34723420343D3420343134303419
:100410003134313462340D340A3400340A108A1411
:100420000A11820745346E34643420346F346634E4
:100430002034503472346F346734723461346D3424
:100440000D340A3400340A108A140A118207453424
:10045000723472346F347234203469346E34203420
:10046000443431343234573472346934743465343A
:10047000283429342C34203475346E346B346E3483
:100480006F3477346E342034743479347034653496
:100490003A342034303478342534783421340D34EF
:1004A0000A3400340A108A140A1182074534783459
:1004B000703465346334743469346E346734203492
:1004C0006F346E34653420346F3466343A340D340E
:1004D0000A340934203430347834253478340D34F7
:1004E0000A34093430347834253478340D340A34FD
:1004F00000340A108A140A11820707340D340A34B2
:100500000D340A341B345B3431343B3433343134EE
:100510006D3449346E3474346534723472347534E5
:100520007034743421341B345B3430343B34333412
:1005300037346D340D340A3400340A108A140A1129
:10054000820743344D3444343A3420342034523416
:10055000653461346434203449346E347434653421
:1005600072347234753470347434203452346534D7
:100570006734693473347434653472340D340A3436
:1005800000340A108A140A11820749346E34743414
:100590006534723472347534703474342034723487
:1005A0006534673469347334743465347234203498
:1005B0006234793474346534733420347734653478
:1005C000723465342034303478342534783420342F
:1005D00061346E34643420343034783425347834E3
:1005E0002E340D340A340D340A3400340A108A14BF
:1005F0000A11FD3E03188A0A820043344D34443404
:100600003A34203420345234653461346434203434
:100610004C3461347334743420345434723461345F
:100620006E34733461346334743469346F346E34CB
:100630002034533474346134743475347334203456
:1006400052346534673469347334743465347234C5
:1006500020342834303478342534783429340D3437
:100660000A3400340A148A140A11820709345334F4
:10067000743461347434753473343A34203430341F
:100680007834253478342E340D340A3400340A1486
:100690008A140A1182075034723465347334733407
:1006A0002034613420346B3465347934203474342C
:1006B0006F34203472346534733475346D3465347A
:1006C0000D340A340D340A34003436308400000806
:1006D0000319792B0130F800F701F70B6D2BF80B9C
:1006E0006C2B4A30F700F70B732B00000000800BD7
:1006F0006A2B0034B91B8D2B0F30F700380EF7052D
:100700000A3077020318872B3030F707892B390816
:10071000F70777080C1E8A2B99000F30B8050A30AE
:1007200038020318952B3030972BB9133908B807C6
:1007300038080C1E992B990000343408F700F7088C
:100740000319A72B013077020319A72BCC2B0030FC
:1007500083168800861083128614340BB42B8316FC
:10076000061383120617B82B83160613831206137B
:10077000350888000130B600652383160611831200
:1007800006118316061183120615340BCB2B831624
:10079000061383120613162CB60136082322B60A56
:1007A000F70077080C1ED22B990025303602031D66
:1007B000CD2B3408B8005730B9007A2321300C1EF5
:1007C000DF2B99000D300C1EE32B99000A300C1E14
:1007D000E72B9900B60136085222B60AF7007708CF
:1007E0000C1EF02B990017303602031DEB2B013045
:1007F000B8005730B9007A231930B70037085222B1
:10080000B70AF70077080C1E032C99001E30370238
:10081000031DFE2BB8015730B9007A230D300C1E92
:100820000F2C99000A300C1E132C99000034FF3055
:10083000831688008312B5013408350203182F2C63
:100840008316861083128610330835078400080843
:1008500080008316861083128614B50A1C2C00347F
:10086000B30133087922B30AF70077080C1E362C3F
:1008700099001F303302031D312CB30133089D2230
:10088000B30AF70077080C1E432C99001F3033027F
:10089000031D3E2C0130B400F430B5009D233030F0
:1008A000B3000230B4001724B3013308C122B30AE5
:1008B000F70077080C1E5A2C990020303302031DD4
:1008C000552C3008B8005730B9007A232230B400D4
:1008D0003408C122B40AF70077080C1E6D2C990069
:1008E00029303402031D682C3108B8005730B90094
:1008F0007A232B30B5003508C122B50AF7007708F6
:100900000C1E802C990030303502031D7B2C8C1E70
:10091000872C1A08B2013208053C031CDD2C40303C
:100920003207B300B4013408F622B40AF70077089E
:100930000C1E982C99002F303402031D932C330881
:10094000B8005730B9007A2329300C1EA52C990025
:100950000D300C1EA92C99000A300C1EAD2C9900EC
:1009600040303207B3000130B4003308B5009D2396
:100970003030B3000130B4001724B3013308322300
:10098000B30AF70077080C1EC32C99000B30330212
:10099000031DBE2C3008B8005730B9007A232E3022
:1009A0000C1ED02C99000D300C1ED42C99000A304E
:1009B0000C1ED82C9900B20A8B2CB30133084723A4
:1009C000B30AF70077080C1EE32C990019303302A4
:1009D000031DDE2C8C1EEA2C1A088B108A110A12B9
:1009E0001D2884011F308305063083169F001930AF
:1009F00099002630980090308312980029108316B1
:100A0000861383128613291C252DAA012A08332058
:100A1000AA0AF70077080C1E0B2D99000E302A0247
:100A2000031D062D0430AA00A8018B1BA8178B13E9
:100A3000FA30B6006523A81B8B17AA0B142D83165A
:100A40008613803083128606032DAA012A084620C9
:100A5000AA0AF70077080C1E2B2D990004302A02F1
:100A6000031D262DAA012A084F20AA0AF70077089D
:100A70000C1E382D990031302A02031D332D013010
:100A80008316860000308800FF30831288008316AA
:100A90008610831286148316061183120615831698
:100AA0008612831286128316061383120613831688
:100AB0000612831206120B138B138B1B5C2D8316ED
:100AC000011383120B168B10C0308B043130AA0037
:100AD0003D300C1E692D9900AA0B682D0D300C1E9F
:100AE0006F2D99000A300C1E732D9900AA012A0857
:100AF0008520AA0AF70077080C1E7C2D99002A3061
:100B00002A02031D772D8C1E832D1A088316861248
:100B100083128616A8018B1BA8178B130130B60011
:100B20006523A81B8B17AA012A08B420AA0AF7007C
:100B300077080C1E992D99001A302A02031D942D56
:100B4000A8018B1BA8178B130130B400D030B5005F
:100B50009D23A81B8B17AA012A08D320AA0AF700F5
:100B600077080C1EB12D990022302A02031DAC2DEE
:100B7000A8018B1BA8178B13B4018030B5009D23EF
:100B8000A81B8B17AA012A08FA20AA0AF7007708DF
:100B90000C1EC82D99001B302A02031DC32DA8016D
:100BA0008B1BA8178B130130B400D830B5009D23E0
:100BB000A81B8B17AA012A081E21AA0AF70077088A
:100BC0000C1EE02D990017302A02031DDB2DA80111
:100BD0008B1BA8178B13B4010130B5009D23A81BF4
:100BE0008B17AA012A083A21AA0AF70077080C1ED7
:100BF000F72D990010302A02031DF22DA8018B1B3E
:100C0000A8178B130130B400F330B5009D23A81B47
:100C10008B17AA012A084F21AA0AF70077080C1E91
:100C20000F2E990025302A02031D0A2EAA012A0838
:100C30007921AA0AF70077080C1E1C2E99001D3096
:100C40002A02031D172EA8018B1BA8178B13B401B2
:100C50001E30B5009D23A81B8B17AA012A089B21D3
:100C6000AA0AF70077080C1E332E99002A302A02B0
:100C7000031D2E2EAA012A08CA21AA0AF700770806
:100C80000C1E402E990014302A02031D3B2EAA018F
:100C90002A08E321AA0AF70077080C1E4D2E9900B6
:100CA00023302A02031D482EA8018B1BA8178B1383
:100CB000B4010B30B5009D23A81B8B17AA012A088D
:100CC0000E22AA0AF70077080C1E642E9900103035
:080CD0002A02031D5F2E6300E0
:02400E00F13F80
:00000001FF
